:100000000BC023C022C021C020C01FC01EC01DC005
:100010001CC01BC01AC0E0C011241FBECFEDCDBF55
:1000200010E0A0E6B0E0E8E4F2E003C0C895319645
:100030000D92AC39B107D1F710E0ACE9B0E001C0E6
:100040001D92AD39B107E1F718C0DACFE82F8E3134
:1000500070F488E388BBFF27AE2FBF2FA258BF4F95
:100060008C918BBBE05AFF4F808188BB089580EE56
:100070008BBB88E388BB08950895CFEDD0E0DEBF49
:10008000CDBF88249EE1992EBB9ABC9ABD9AD09A86
:10009000D19AD29AD39AD49AD59AD69AD79A63D02B
:1000A000BE98C69884E04BD0882D4ED000E010E07A
:1000B000C0E0D0E08C2FCADF2196CE31D105D4F339
:1000C0000F5F1F4F83E0083E180794F3AA24BB2458
:1000D0008EE1C82ED12C89E063D0082F192F882DEE
:1000E000B5DF89E05DD0E82EF92E892DAFDF89E0FC
:1000F00057D0080F191F912F802F8E0D9F1D63E081
:1001000070E079D0972F862F805092406DE070E09C
:1001100072D0D72FC62F2F968C2F98DFAC16BD0626
:100120002CF48C2EAC2EBB24A7FCB094CC15DD0592
:1001300094F69C2ECC2EDD24C7FCD094CCCF96B167
:10014000987F982B96B9089527B12F73992700248B
:10015000969587950794969587950794982F802D67
:10016000282B27B90895379A359886E0E8DF81E093
:10017000EBDF3D98339A10929C0078940895339861
:100180003798089597B1907E8F71982B97B90895FD
:10019000349A369A089586B199278074907008959C
:1001A00010929C0097B1907E8F71982B97B9349ADA
:1001B000369A3699FECF84B1282F332785B19927F7
:1001C000982F8827822B932B0895EADF96958795A1
:1001D00096958795992708951F920F920FB60F92C3
:1001E00011248F9381E080939C008F910F900FBE1C
:1001F0000F901F90189597FB092E07260AD077FDC0
:1002000004D00CD006D000201AF4709561957F4F71
:100210000895F6F7909581959F4F0895AA1BBB1BF3
:1002200051E107C0AA1FBB1FA617B70710F0A61BF6
:10023000B70B881F991F5A95A9F780959095682F3D
:08024000792F8A2F9B2F0895EE
:10024800383838383838383838383838383838302E
:100258003030303028282828281818181818C1C213
:10026800C4C8D0A1A2A4A8B06162646870E1E2E445
:0C027800E8F0E1E2E4E8F0E1E2E4E8F0A4
:00000001FF
